:100000000C945F000C94D9000C94D9000C94D90086
:100010000C94D9000C944C100C94D9000C94D90079
:100020000C94D9000C94D9000C94D9000C94D900EC
:100030000C94D9000C94D9000C94D9000C94290A82
:100040000C94D9000C94D9000C94340F0C94980F94
:100050000C94D9000C94D9000C94D9000C94D900BC
:100060000C94D9000C94D9000C94D9000C94D900AC
:100070000C94D9000C94D9000C94D9000C94D9009C
:100080000C94D9000C94D9000C94D900E116EB160D
:10009000F216F81602171017DE16DE16DE16DE163A
:1000A0001F17251728173A173D174817DE164B1745
:1000B000511754175A175D17631766176E1785B7D0
:1000C000806885BFECE6F0E0808180688083BF9A1D
:1000D000BE9AC798C69880EC85BFAF9AA79AAE9A89
:1000E000A69A81EE8093008380E48093018385B794
:1000F0008F7785BF80E090E09D9B05C0019641F021
:100100009D9BF8CFFBCF019619F09D99F3CFFBCFC4
:1001100085B7806885BFAF98A798AE98A69887E006
:1001200089B98093990011241FBECFEFD0E1DEBFC3
:10013000CDBF11E0A0E0B1E0EEE1F7E300E00BBFDE
:1001400002C007900D92AA3DB107D9F712E0AAEDBF
:10015000B1E001C01D92A333B107E1F78FEF9FEF2C
:100160009EBF8DBF23E332E0C901809590958158F1
:10017000914038F06FEF7EEF621B730BC9010E9454
:10018000C6060E940007892B41F06BE171E087E011
:1001900092E00E940C1B0E94E70620E831E040E05C
:1001A00050E065E671E084E291E00E94C5080C949D
:1001B00000000C940000EF92FF920F931F93CF93D7
:1001C000DF93CDB7DEB764970FB6F894DEBF0FBEEE
:1001D000CDBF8091F2019091F3010E94721044E131
:1001E00050E08E010F5F1F4FB8010E944D117C013E
:1001F0000E94291321E041E060E085E00E94861220
:100200002FEF44E060E087E00E9486128091F201C7
:100210009091F3010E947210A701B8010E94601131
:10022000D8CF0F931F93CF93DF93CDB7DEB724972B
:100230000FB6F894DEBF0FBECDBF80E09BE4A0E018
:10024000B0E089839A83AB83BC830E94081205E3E4
:1002500011E040E060E070E0C8010E94AA0160E0A7
:1002600071E0C80102960E9476109093F30180938A
:10027000F2010E947210AE014F5F5F4F61E071E0CA
:100280000E94E3106091F2017091F30183E091E02C
:100290000E94D21081E00E9432132FEF44E060E010
:1002A00087E00E9486120E94DB0081E090E02496A5
:1002B0000FB6F894DEBF0FBECDBFDF91CF911F9177
:1002C0000F91089580932E0108950E946B0220E003
:1002D00033E040E050E061E171E089E291E00E94AA
:1002E000C5088EEF0E944A050E94CE050E941505A2
:1002F00020912E012F3FC1F395B785B7837E822BC6
:1003000085BF85B7806285BF889585B78F7D85BF9E
:1003100085B7837E9C71892B85BFE6CF0F931F9392
:10032000CF93DF938C01C091DB01D091DC010AC037
:10033000B801CE0102960E94021B892B29F0099078
:10034000D881C02D2097A1F7CE01DF91CF911F91C9
:100350000F910895CF93DF93EC01892B11F1611573
:10036000710511F07D876C8741114E87CE01029691
:100370000E948E01892BA9F4EB89FC89309721F02A
:10038000CE010995892B69F48091DB019091DC0104
:1003900099838883D093DC01C093DB0180E090E0F7
:1003A00002C08FEF9FEFDF91CF9108958091F6010A
:1003B0009091F701A091F801B091F9010196A11D6A
:1003C000B11D8093F6019093F701A093F801B093CB
:1003D000F9010895CF93DF93EC011B821A82E0911B
:1003E000F401F091F5011AC0288539854A855B85AD
:1003F00080859185A285B385281739074A075B0751
:1004000080F0281B390B4A0B5B0B288739874A87FA
:100410005B87FB83EA830190F081E02D309721F721
:1004200018C0821B930BA40BB50B80879187A28702
:10043000B387F983E883D383C283EA81FB81309752
:1004400019F0D183C08308C0D093F501C093F401A3
:1004500003C019821882F1CFDF91CF9108950FB6B2
:10046000F8940F926091F6017091F7018091F80174
:100470009091F9010F900FBE0895CF93DF93EC0197
:10048000EA81FB8188819981309719F0918380837B
:1004900004C09093F5018093F401E881F9813097CD
:1004A000A1F08A819B819383828380859185A28537
:1004B000B385288539854A855B85820F931FA41FE4
:1004C000B51F80879187A287B387CE010E94590606
:1004D000DF91CF91089586ED91E00E947F0987B763
:1004E000826087BF0895EF92FF920F931F93CF937F
:1004F000DF930FB6F8940F922091F6013091F70137
:100500004091F8015091F9010F900FBE8091DD01EB
:100510009091DE01A091DF01B091E00179018A01A3
:10052000E81AF90A0A0B1B0B2093DD013093DE0158
:100530004093DF015093E0014FC088859985AA85DB
:10054000BB85E816F9060A071B07A0F48E199F0958
:10055000A00BB10B88879987AA87BB870097A10555
:10056000B10521F0EE24FF24870136C0EE24FF24DC
:10057000870108C0E81AF90A0A0B1B0B18861986AE
:100580001A861B86EC85FD85309721F06E857F8568
:10059000CE0109958C819D81AE81BF818887998725
:1005A000AA87BB870097A105B10521F4CE010E945F
:1005B0003D0212C0E091F401F091F5010190F0814B
:1005C000E02DF093F501E093F401309711F01382E0
:1005D0001282CE010E94EA01C091F401D091F5018E
:1005E000209731F0E114F1040105110509F0A5CFC0
:1005F000DF91CF911F910F91FF90EF9008952F926F
:100600003F924F925F926F927F928F929F92AF92A2
:10061000BF92CF92DF92EF92FF920F931F93CF93EF
:10062000DF93CDB7DEB724970FB6F894DEBF0FBEC9
:10063000CDBF0FB6F8940F92A090F601B090F701DD
:10064000C090F801D090F9010F900FBE0E947A0976
:100650009B01AC01C601B5010E94451B39014A014D
:100660000E947A091B012C010E947A0969837A830E
:100670008B839C83C401B30128EE33E040E050E05B
:100680000E94131B7B018C01C401B301A2019101E3
:100690000E94131BA61AB70AC80AD90AC601B501D7
:1006A00028EE33E040E050E00E94131B29813A819C
:1006B0004B815C810E94451BE20EF31E041F151F37
:1006C000C801B70124960FB6F894DEBF0FBECDBFA8
:1006D000DF91CF911F910F91FF90EF90DF90CF901E
:1006E000BF90AF909F908F907F906F905F904F9052
:1006F0003F902F900895EF92FF920F931F930FB6A4
:10070000F8940F92E090F601F090F7010091F80153
:100710001091F9010F900FBE0E947A099B01AC0164
:10072000C801B7010E94451BCA01B9011F910F9171
:10073000FF90EF900895AF92BF92CF92DF92EF9229
:10074000FF920F93CF93DF936B017C01EA01590174
:1007500080E190E00E94E605FC01892B81F10FB653
:10076000F8940F928091F6019091F701A091F80111
:10077000B091F9010F900FBE8C0D9D1DAE1DBF1DD8
:100780002091DD013091DE014091DF015091E001C7
:10079000821B930BA40BB50B80879187A287B3872D
:1007A00000FF05C0148215821682178204C0C4821D
:1007B000D582E682F782D587C487B786A686CF0121
:1007C000DF91CF910F91FF90EF90DF90CF90BF908E
:1007D000AF9008950F93CF93DF930E949B03EC019A
:1007E000009711F00E94EA01CE01DF91CF910F91A5
:1007F0000895CF92DF92EF92FF920F936A017901F1
:100800000E94CF099701A6010E94EA030F91FF9071
:10081000EF90DF90CF900895AF92BF92CF92DF928A
:10082000EF92FF920F93CF93DF935B016C01611501
:10083000710581059105D1F1CCEFD1E0BE01809128
:10084000FE019091FF010E94B004E091FE01F09141
:10085000FF0183E08787E090FE01F090FF0101E057
:1008600097014BEE54E0C601B5010E94F903F70170
:10087000968B858B892B19F00E94890519C0E09110
:10088000FE01F091FF01D08FC78B8091FC01909108
:10089000FD019383828381E087878091FE0190919F
:1008A000FF019093FD018093FC0102C00E94CE05E0
:1008B000DF91CF910F91FF90EF90DF90CF90BF909D
:1008C000AF900895CF93DF93DC019B01EC01788F0B
:1008D0006F8B1D821C820FB6F8940F92EB01E8819A
:1008E000F9818FEFEF3FF80749F4ED018C819D818D
:1008F00001969D838C83E0E0F0E015C0309799F07D
:100900000F900FBEED019A8908C09F012E5F3F4FE7
:100910000280F381E02D309719F082899817A8F7AB
:100920000FB6F8940F92ED01FB83EA83F901B183CE
:10093000A083EA81FB81309771F084819581892BB6
:1009400051F08C819D8124813581820F931F9D837D
:100950008C83158214820F900FBEDF91CF91089582
:10096000CF93DF939C01DB010FB6F8940F92ED91CA
:10097000FC9111970F900FBE8FEFEF3FF80731F505
:1009800027C082819381E217F307E9F40FB6F89448
:100990000F9211969C938E9384819581892B59F0A7
:1009A000A281B381109729F084819581ED019D8307
:1009B0008C83158214820F900FBEF901138212826C
:1009C000108E178A05C0DF011296FC013097C9F618
:1009D000DF91CF910895FB01168A158A82E08787FF
:1009E0006CEF71E0CF010E94620408950F931F9392
:1009F000CF93DF938C01C091FA01D091FB010CC021
:100A0000B801CE0106960E94021B892B11F4CE017B
:100A100007C00990D881C02D209791F780E090E021
:100A2000DF91CF911F910F910895E0910002F09115
:100A30000102309741F0838994890E9459061092EF
:100A40000102109200020895CF93DF93C091FA0142
:100A5000D091FB010E9415052091FE013091FF010C
:100A6000EAEFF1E00AC088819981C217D30719F42F
:100A70009183808304C0FE01EC012097A1F780914F
:100A8000FE019091FF019093010280930002DF919B
:100A9000CF9108950F931F93182FE091FE01F091CD
:100AA000FF0102896CEF71E0CF010E94B004E09178
:100AB000FE01F091FF01128B1F3F49F06CEF71E0D6
:100AC0008091FE019091FF010E94620402C00E9489
:100AD0002405E091FE01F091FF018091FC019091CD
:100AE000FD01E817F90719F481E0878709C082E062
:100AF00087870FB6F8940F920E9486080F900FBE5A
:100B0000802F99271F910F9108958FEF0E944A051A
:100B10000895CF93DF93C091FA01D091FB0120C0DB
:100B20000FB6F8940F928C819D810F900FBE892B88
:100B3000A1F0EF89F88D0FB6F8940F928C819D810A
:100B400001979D838C830F900FBE808191818F5F71
:100B50009F4F19F0CF010E941C070990D881C02D2A
:100B60002097F1F60E947302E091FE01F091FF01DF
:100B70008091FC019091FD01E817F90761F08785EC
:100B8000813011F482E087870FB6F8940F920E94AB
:100B900086080F900FBEDF91CF910895E091FE017E
:100BA000F091FF0182819381892B69F06CEF71E0F4
:100BB000CF010E94B0046CEF71E08091FE01909132
:100BC000FF010E9462040E94890508950F931F93FC
:100BD000CF93DF930091E1011091E201801791071B
:100BE00030F080E090E060C0EF01DB012FC0AC018D
:100BF0004A5F5F4F4430510510F444E050E0E0910B
:100C00000202F091030262E072E0C0E0D0E0A0E0F6
:100C1000B0E017C0208131812417350760F0241718
:100C2000350711F3209729F0888199812817390712
:100C300010F4EF01DB01BF016E5F7F4F0280F38193
:100C4000E02D309739F7CE01209771F12881398155
:100C5000CA010A966A817B818217930770F4FE01AC
:100C6000E40FF51F241B350B3183208373836283CC
:100C700059834883ED93FC9302C06D937C93E88184
:100C8000F9810E1B1F0B1093E2010093E101EC0FA1
:100C9000FD1F34978FEE9EEBADEABEED808391830E
:100CA000A283B383CE010296DF91CF911F910F9162
:100CB0000895CF93DF93DC0112976D917C9111978A
:100CC000E0910202F0910302C2E0D2E03AC040811A
:100CD0005181CF01840F951F8A179B07C1F49A0198
:100CE000260F371F3183208382819381DF01A20F7A
:100CF000B31FA817B90791F58D919C911197280FF3
:100D0000391F31832083ED018A819B8125C0AE1775
:100D1000BF0778F4B983A8832D913C911197CD0139
:100D2000820F931F8E179F0779F0ED01FB83EA83F3
:100D300015C0A817B90728F1EF0122960280F381A8
:100D4000E02D309721F617C0240F351F11963C93E4
:100D50002E9382819381FD01938382838091E101AF
:100D60009091E201860F971F9093E2018093E10139
:100D700080E090E008C0FD0113821282B983A8834D
:100D8000EDCF8FEF9FEFDF91CF910895FC0161933D
:100D90007193CF010E94590608958091E1019091CD
:100DA000E20108950F931F93CF93DF938C010E946C
:100DB000E605EC01009729F0A80160E070E00E94D0
:100DC000F81ACE01DF91CF911F910F91089583E121
:100DD000809304028FE48093050283E580930602EA
:100DE00043E150E064E072E080E090E00E94780827
:100DF000892B19F08FEF9FEF089580E090E0089520
:100E000043E150E064E072E080E090E00E947B0803
:100E1000892B79F480910402833159F48091050281
:100E20008F3439F480910602833519F480E090E024
:100E300008958FEF9FEF0895CF93DF93DC010FB6F6
:100E4000F8940F92CD91DC9111970F900FBE8FEF18
:100E5000CF3FD80709F43AC0209771F10FB6F89444
:100E60000F92EA81FB811196FC93EE938C819D8118
:100E7000892B71F0309729F08C819D819583848333
:100E800005C08FEF9FEF11969C938E931D821C825D
:100E90000F900FBE8D899E89009721F00E943D0220
:100EA0001E8A1D8A82E08F876CEF71E0CE010E945E
:100EB000620481E090E00CC00FB6F8940F928FEFBF
:100EC0009FEF11969C938E930F900FBE80E090E061
:100ED000DF91CF9108950F931F93CF93DF93EC0190
:100EE0000FB6F8940F92888199810F900FBE2FEF63
:100EF0008F3F920741F40FB6F8940F92198218822F
:100F00000F900FBE02C0892B19F400E010E012C050
:100F100000E010E0CE010E941C07080F191F0FB659
:100F2000F8940F92888199810F900FBE01978E5F80
:100F30009F4F80F3C801DF91CF911F910F910895CA
:100F40000F931F930E946B078C010E94CE05C8016E
:100F50001F910F9108950F931F930E941C078C01FE
:100F60000E94CE05C8011F910F910895CF93DF9382
:100F7000AC01DB010FB6F8940F92CD91DC91119783
:100F80000F900FBE8FEFCF3FD80799F534C08D89F2
:100F90009E892A813B818417950741F50FB6F89405
:100FA0000F9211963C932E938C819D81892B81F019
:100FB000EA81FB81309729F08C819D819583848320
:100FC00005C08FEF9FEF11969C938E931D821C821C
:100FD0000F900FBE82E08F876CEF71E0CE010E9410
:100FE00062048FEF9FEF9E8B8D8B05C0DE01129602
:100FF000E901209761F6DF91CF910895AF92BF92FA
:10100000CF92DF92EF92FF920F93CF93DF93EC0199
:101010005A016B010FB6F8940F92888199810F9055
:101020000FBE8F5F9F4F51F40FB6F8940F92198245
:1010300018820F900FBE0E94CE0538C06CEF71E091
:101040008091FE019091FF010E94B004BE01809149
:10105000FE019091FF010E946204E091FE01F09177
:10106000FF0183E08787E090FE01F090FF01A1146B
:10107000B104C104D10461F001E09E0146EB57E0E8
:10108000C601B5010E94F903F701968B858B03C059
:10109000F701168A158A0E948905E091FE01F091F8
:1010A000FF01858996898F5F9F4F19F080E090E05E
:1010B00004C0168A158A8FEF9FEFDF91CF910F91B1
:1010C000FF90EF90DF90CF90BF90AF900895FC011C
:1010D0000FB6F8940F92808191818F5F9F4F11F42A
:1010E000118210820F900FBECF010E94FE0708955B
:1010F0000E94BE0E08950E94DE0E08959F918F916A
:101100000F900BBE0F900FBE1F9018952F923F921D
:101110004F925F926F927F928F929F92AF92BF9207
:10112000CF92DF92EF92FF920F931F93CF93DF93B3
:101130008DB79EB7E091FE01F091FF01918B808BFE
:10114000E091FC01F091FD01F093FF01E093FE01BD
:1011500081E08787E091FE01F091FF01808991890C
:101160008DBF9EBFDF91CF911F910F91FF90EF90A8
:10117000DF90CF90BF90AF909F908F907F906F90B7
:101180005F904F903F902F900895CF92DF92EF9213
:10119000FF920F931F93CF93DF938C017B016A0122
:1011A000E901C90149960E94E605FC01009719F47E
:1011B00080E090E075C0C80FD91F9E0127503040D5
:1011C000AE014B515040CE01069668E0D8010D901B
:1011D0008D01DC010D92CD016150C1F71E86415099
:1011E0005040598B488B4F5F5F4FFC8BEB8B8FEEE2
:1011F0009EEBADEABEED80839183A283B3838483AB
:101200009583A683B78380879187A287B3878487D6
:101210009587A687B78780E48A8B8F2D9927F90158
:101220008583E68280E8838312821482C1828D2DB9
:10123000992780832EE738E0832F9927FA01828B44
:10124000238B8091FA019091FB0199838883D0933D
:10125000FB01C093FA0112E01F871E8A1D8A188EB7
:101260001F8A6CEF71E0CE010E946204E091FE01E2
:10127000F091FF01309721F40FB6F8940F9260CFF0
:101280008091FC019091FD01E817F90741F0178763
:101290000FB6F8940F920E9486080F900FBECE01F1
:1012A000DF91CF911F910F91FF90EF90DF90CF9042
:1012B00008951F93182F6091E3017091E4018091CC
:1012C000E5019091E60120EA3FE040E050E00E9415
:1012D000451B822F932F0197F1F71A95D1F71F9194
:1012E00008956091E3017091E4018091E50190918E
:1012F000E601089560E074E080E090E00895BC01AC
:1013000087B78D7F87BF80B7886080BF12BE82E0BD
:1013100083BF80B7992787709070892BD1F781E0C0
:1013200086BF0FB6F8940F9281E090E0A0E0B0E0A5
:10133000B6B7B170E9F3B6BF0894811D911DA11D28
:10134000B6B7B170C9F3BB270F900FBE27E0880F67
:10135000991FAA1FBB1F2A95D1F78093E301909391
:10136000E401A093E501B093E60187B78D7F87BFC5
:1013700080B7886080BF12BE89E083BF8FE181BFE4
:1013800080B7992787709070892BD1F782E086BF4C
:1013900040E050E08FE291E00E94151A089528EE97
:1013A00033E040E050E00E94131B3AE096958795A9
:1013B000779567953A95D1F708959C01FB0187B71A
:1013C000482F55274270507087B78D7F87BF2031D7
:1013D0003105D9F0213131053CF42115310581F079
:1013E0002130310551F40EC02231310571F1223125
:1013F0003105E4F020323105E1F02FEF3FEF1FC05F
:1014000040E050E082E086BF18C006B601FE05C08D
:1014100081E090E09183808302C011821082452B8D
:10142000A1F08081918180689183808320E030E009
:1014300008C08EE090E09183808320E030E0452B6F
:1014400031F087B7826087BF02C020E030E0C90179
:1014500008951F920F920FB60F9211242F933F936E
:101460004F935F936F937F938F939F93AF93BF93AC
:10147000EF93FF938FE291E00E94071AFF91EF91A3
:10148000BF91AF919F918F917F916F915F914F919C
:101490003F912F910F900FBE0F901F901895559A66
:1014A00089B78F7E89BF0895CF93DF93DC01EC016C
:1014B000EA81FB812091E801422F5527CA01807300
:1014C0009070892B89F044FF04C083E18CB92064BB
:1014D00003C081E18CB92F7B2093E8018091E80162
:1014E0008F7C8093E80155C027FF02C0559851C0FA
:1014F000ED018A859B85892BB1F18091EB018823D1
:1015000039F00C9B05C0559889B7806189BF41C0EF
:10151000ED018A859B8501979B878A878091E901E8
:10152000882311F0509A01C0509881918CB99F0185
:10153000FD01868197812817390711F424813581AF
:10154000ED013B832A832A853B858C859D85281761
:101550003907F9F4E889F989309769F08FEFEF3F9F
:10156000F807B9F011C05598ED011B861A86E88975
:10157000F989309729F48FEF9FEF998B888B09C0F9
:101580008FEFEF3FF80729F08481958101969583CD
:101590008483DF91CF910895CF93DF93DC013BB13A
:1015A0008091E701382B3093E7016CB12091E8017D
:1015B000222361F0633119F45598206804C0613129
:1015C00029F4559A2F772093E8015DC0ED014A85F3
:1015D0005B85888599854817590720F038603093D6
:1015E000E70151C04F5F5F4F41305105A1F4ED015C
:1015F000E889F989309729F48FEF9FEF998B888BD1
:101600002AC08FEFEF3FF80731F184819581019671
:101610009583848320C0222399F0ED018E859F85D8
:1016200048175907C0F026FD16C05D9B05C083E131
:101630008CB920642F7D01C020622093E8010BC08B
:101640008091EA01882339F0FD0186859785481746
:10165000590708F01A9AED91FC9111976193119630
:10166000FC93EE932D913C911197ED018E819F811A
:101670002817390729F48C819D8111969C938E93AC
:10168000FD0153874287DF91CF910895529B03C09C
:1016900089E090E008958091950082FF0AC08091D2
:1016A000950081FF03C088E090E0089587E090E016
:1016B00008958091950081FF03C086E090E0089531
:1016C00085E090E008958091950085FD03C080E05D
:1016D00090E008958091950084FF03C081E090E040
:1016E000089582E090E008958091950083FF03C003
:1016F00082E090E0089581E090E00895EF92FF92FB
:101700000F931F938091E701682F7727CB0174E037
:10171000969587957A95E1F79C0144275527217086
:1017200030704070507063FD226062FD24608091D3
:10173000E801882321F086FD426087FD48601A9BFE
:1017400014C0E12C62E0F62E012D112DE22AF32ABD
:10175000042B152B8091EA01882381F0E12C92E083
:10176000F92E92E0092F112D05C0E12C81E0F82E11
:10177000012D112DE22AF32A042B152B0C9B0CC0F2
:10178000A801970138608091EB01882341F0A801FE
:1017900097013860426003C0A8019701346041FF9F
:1017A000416043FF44608091E901882321F0CA0130
:1017B000B901806403C0CA01B9018068589B02C0A6
:1017C000806101C080621F910F91FF90EF9008959A
:1017D000EF92FF920F931F937B018C018091E801A0
:1017E0008823D9F00FB6F8940F9200FF02C08F7BC8
:1017F00003C001FF03C080648093E80102FF04C0BE
:101800008091E8018F7705C003FF05C08091E80152
:1018100080688093E8010F900FBE8091EA018823D1
:1018200021F001FD1A9A00FD1A98F1FC1A9AF0FCB9
:101830001A9806FF03C081E08093E90107FF02C008
:101840001092E90104FD589A05FD5898E0FE05C084
:101850008091E7018F7E8093E701E1FE05C08091D2
:10186000E701877F8093E701E2FE05C08091E701F1
:101870008B7F8093E7010E947E0B687F6E157F054A
:101880008007910719F08FEF9FEF02C080E090E092
:101890001F910F91FF90EF9008958091950086FF22
:1018A0000BC0129B02C093E001C091E080919500B3
:1018B00080FF07C0946005C0599B02C090E201C040
:1018C00090E0892F992708958091E801882329F0D5
:1018D00020E230E040E050E004C020E030E040E0B2
:1018E00050E08091EA01882311F0216001C02E7F31
:1018F0008091EB01882321F0CA01B901626008954B
:10190000CA01B9016D7F0895559A08959091E80133
:101910009923A9F096FF13C00FB6F8940F925D9B20
:1019200004C081E18CB99F7E01C090619093E80171
:101930008091E8018F798093E8010F900FBE80912C
:10194000EA0181111A9808950FB6F8940F925798EA
:10195000569855980F900FBE8AE00E9459095498E6
:10196000539808951F93182F0E94A40C52988091A9
:1019700095008D7F80939500809195008B7F80935B
:1019800095001730A1F0183018F41630A9F405C0EE
:10199000183041F0193081F404C0809195008260C4
:1019A00009C0529A80919500826080939500809141
:1019B00095008460809395000FB6F8940F9288EBA1
:1019C0008AB90F900FBE0E94460B811719F08FEF56
:1019D0009FEF02C080E090E01F9108958F929F9248
:1019E000AF92BF92CF92DF92EF92FF920F931F932D
:1019F00089B0909090008091950086FF06C0B2E07B
:101A0000AB2EB12CC12CD12C0DC0599B06C0A8E027
:101A1000AA2EB12CC12CD12C05C0F0E1AF2EB12CD7
:101A2000C12CD12C0E9471097B018C01282D3327F8
:101A3000892D9927982F8827282B392B442755271C
:101A40002F5F3F4F4F4F5F4FC601B5010E94131BE1
:101A50009B01AC01C801B7010E94451BCA01B90135
:101A60001F910F91FF90EF90DF90CF90BF90AF90BC
:101A70009F908F90089540E050E060E070E081EB2F
:101A800091E00E94151A40E050E060E070E087EBC2
:101A900091E00E94151A8091EB01882359F0109271
:101AA000EB01149840E050E060E070E08DEB91E0D5
:101AB0000E94151A8091EA01882319F01092EA0118
:101AC000129880E090E008954AE751E06CEC7AE0EB
:101AD00081EB91E00E94151A892B19F08FEF9FEF8F
:101AE000089548E651E064E57AE087EB91E00E94D2
:101AF000151A892B19F480E090E0089540E050E039
:101B000060E070E081EB91E00E94151A8FEF9FEF8B
:101B10000895EF92FF920F931F937B018C0165FF55
:101B20000BC08091E801882371F40FB6F8940F92EE
:101B300081E48093E80105C00FB6F8940F921092EB
:101B4000E8010F900FBEE0FE06C01A9A129A81E0DB
:101B50008093EA0107C08091EA01882319F010926E
:101B6000EA011298E1FE10C040E050E06FE47AE034
:101B70008DEB91E00E94151A892BF9F41C9A1498A8
:101B800081E08093EB010FC08091EB01882359F035
:101B90001092EB0140E050E060E070E08DEB91E0EE
:101BA0000E94151A14980E94640C6E157F05800718
:101BB000910719F480E090E002C08FEF9FEF1F9132
:101BC0000F91FF90EF900895EF92FF920F931F9364
:101BD0007B018C010E94A40C8091950086FD11C0B0
:101BE000599B08C092E0EE0CFF1C001F111F9A9534
:101BF000D1F707C083E0EE0CFF1C001F111F8A9570
:101C0000D1F70E947109A80197010E94451B2F5F1F
:101C10003F4F4F4F5F4F569547953795279521502A
:101C2000304029B9232F3327209390000FB6F89422
:101C30000F9288EB8AB90F900FBE80E090E01F9161
:101C40000F91FF90EF9008951F93182F0E94A40CFE
:101C5000812F992780FF13C081FF02C0129A01C013
:101C6000129882FF04C080919500816003C080912A
:101C700095008E7F8093950059985E9A0FC085FFDE
:101C800002C0599A01C05998809195008E7F809327
:101C90009500809195008F7B809395000FB6F89406
:101CA0000F9288EB8AB90F900FBE0E944D0C8117DE
:101CB00019F08FEF9FEF02C080E090E01F91089530
:101CC0001F93182F0E94A40C113071F0113018F0DE
:101CD0001230C1F40DC0809195008F7E80939500E5
:101CE000809195008F7D0CC080919500806103C02C
:101CF000809195008F7E8093950080919500806201
:101D0000809395000FB6F8940F9288EB8AB90F90E4
:101D10000FBE0E94630B811719F08FEF9FEF02C077
:101D200080E090E01F9108951F93182F0E94A40C4B
:101D3000113021F480919500877F05C0123029F47D
:101D4000809195008860809395000FB6F8940F926B
:101D500088EB8AB90F900FBE8091950083FF03C076
:101D600082E090E002C081E090E0181719F08FEF58
:101D70009FEF02C080E090E01F910895CF93DF9322
:101D8000EA019C0140E050E0FB0110C0D9010E9433
:101D90007B1B802D9081981721F0D901092E0E947C
:101DA000831B4F5F5F4F31962F5F3F4F4C175D078F
:101DB00069F780E090E0DF91CF910895CF93DF93B2
:101DC000EA01DC01FB01219724F00E947B1B0192B8
:101DD000FACF80E090E0DF91CF9108959C01FB0164
:101DE0008AB1482F552740785070579820313105D7
:101DF000D9F0213131053CF42115310581F0213034
:101E0000310551F40EC02231310559F1223131052D
:101E1000DCF020323105D9F08FEF9FEF1EC040E09B
:101E200050E08CB18CB117C05F9B05C081E090E0A1
:101E30009183808302C011821082452B91F08081B2
:101E4000918180689183808380E090E008C080E188
:101E500090E09183808380E090E0452B21F0579AB9
:101E6000089580E090E008951F920F920FB60F92B0
:101E700011242F933F934F935F936F937F938F938F
:101E80009F93AF93BF93EF93FF9381EB91E00E94F9
:101E9000071AFF91EF91BF91AF919F918F917F9121
:101EA0006F915F914F913F912F910F900FBE0F90C7
:101EB0001F9018959C01FB018AB1482F552740724D
:101EC000507055982131310519F1223131053CF41A
:101ED0002115310551F12031310539F409C0223184
:101EE000310519F120323105B1F08FEF9FEF19C0A4
:101EF0005D9B05C081E090E09183808302C01182E8
:101F00001082452B91F0808191818068918380833C
:101F100080E090E008C080E190E09183808380E0E1
:101F200090E0452B21F0559A089580E090E00895C7
:101F30001F920F920FB60F9211242F933F934F933E
:101F40005F936F937F938F939F93AF93BF93EF9321
:101F5000FF9387EB91E00E94071AFF91EF91BF91E9
:101F6000AF919F918F917F916F915F914F913F9131
:101F70002F910F900FBE0F901F9018959C01FB01A1
:101F800089B7482F55274071507089B78F7E89BF18
:101F900021313105D1F1223131054CF421303105A7
:101FA000F9F020313105F9F0232BA1F069C0283177
:101FB000310571F1293131052CF42231310509F057
:101FC0005FC066C029313105B9F12032310509F011
:101FD00057C053C08AB78E7F8ABF8AB78D7F8ABFAA
:101FE00080E188BF1EC008B604FE05C081E090E015
:101FF0009183808302C011821082452B09F448C06E
:102000008081918180689183808320E030E03CC0B2
:102010008AB7982F927081FF07C085E090E0918386
:10202000808320E030E02EC0913019F487E090E00A
:10203000F6CF81E090E0F3CF60817181613071056E
:1020400019F48AB78E7F05C06730710531F48AB7FD
:1020500081608ABF8AB78D7F0EC06530710519F423
:102060008AB78E7F05C06630710551F48AB78160EA
:102070008ABF8AB782608ABFD4CF84E090E0CFCF96
:102080002FEF3FEF452B31F089B7806189BF02C048
:1020900020E030E0C90108951F920F920FB60F9211
:1020A00011242F933F934F935F936F937F938F935D
:1020B0009F93AF93BF93EF93FF938DEB91E00E94BB
:1020C000071AFF91EF91BF91AF919F918F917F91EF
:1020D0006F915F914F913F912F910F900FBE0F9095
:1020E0001F901895FC01808191810895CF92DF9215
:1020F000EF92FF920F931F93CF93DF936C01CB016D
:102100000E9483117C018F5F9F4F71F440C00F5F6D
:102110001F4F32960830110559F487E190E09093F3
:1021200032028093310233C003E010E0E9ECF1E0C9
:1021300080819181892B59F787E090E00E94761188
:10214000EC01000F111F0D531E4FD801CD93DC93EE
:102150002097E9F0B701C6010E94F51099838883A2
:10216000D801ED91FC918F5F9F4F39F4CF010E9410
:102170007311F801118210820AC0F382E282148284
:10218000D801ED91FC9116821582CF0102C080E04A
:1021900090E0DF91CF911F910F91FF90EF90DF9032
:1021A000CF900895FC01CB01DF010D900020E9F7ED
:1021B0001197AE1BBF0BAD01BF01FC018081918166
:1021C0000E9460110895CF93DF93EC01AA81BB8137
:1021D000109719F4EB85FC8504C0ED01ED89FE89AB
:1021E000CD010995DF91CF910895EF92FF920F9362
:1021F0001F93CF93DF93CDB7DEB729970FB6F8942F
:10220000DEBF0FBECDBF7B018C01FE013196AE015A
:10221000475F5F4F03C021930F5F1F4F302F381B65
:10222000D8012C91222329F02A3319F0E417F5075D
:1022300091F7CE010196FC01E30FF11D10820E947F
:102240008E01DC01892B49F482E090E09093320208
:10225000809331028FEF9FEF13C0F80180818A33A2
:1022600019F060E070E003C0B8016F5F7F4FFD01BF
:10227000058D168D20E030E0A701CD01F80109950C
:1022800029960FB6F894DEBF0FBECDBFDF91CF9178
:102290001F910F91FF90EF900895CF93DF93DC0192
:1022A000EC01EA81FB81309719F4ED81FE8103C0D6
:1022B0000788F08DE02DCD010995DF91CF9108952C
:1022C000CF93DF93DC01EC01EA81FB81309719F4B5
:1022D000EF81F88503C0018CF28DE02DCD010995C9
:1022E000DF91CF9108950E94590608950E94E60556
:1022F0009C01892B31F48CE090E090933202809322
:102300003102C9010895FC018081823759F0873775
:1023100019F08136B1F403C081E093E41BC088E07A
:1023200091E418C080E090E415C02B3219F02236F9
:1023300041F404C08E7F826093600CC09F7B9068E4
:1023400009C086E190E090933202809331028FEFD2
:102350009FEF089531962081222339F7089508953B
:1023600084B7806884BF84BF089584B78F7784BFA3
:1023700084BF0895EAE9F0E08081877F80838B98AD
:1023800093988A9892988C98949815981D98A1E69D
:10239000B0E08C918F7B8C93E2E6F0E080818F7BC4
:1023A00080838C918F7D8C9380818F7D80838C91B5
:1023B0008F7E8C9380818F7E80830895EAE9F0E0A0
:1023C0008081886080838B9A939A8A98929A8C9A5B
:1023D00015980895882321F084E00E946B120895D7
:1023E00084E00E9478120895882321F085E00E94FD
:1023F0006B12089585E00E9478120895882321F0D9
:1024000087E00E947812089587E00E946B12089579
:10241000189A939A8B9A80E00E946201089588230B
:1024200021F086E00E946B1203C086E00E947812C1
:1024300083ED91E00E94BA1184B7806884BF84BFA5
:1024400008950F931F9303ED11E0C8010E94BA1184
:1024500084B7806884BF84BF80E00E940F1281E04F
:102460000E94FE1168EE73E080E090E00E940C0490
:1024700081E00E940F1264EF71E080E090E00E9422
:102480000C0480E00E94FE1184B78F7784BF84BF64
:10249000C8010E94DE1160ED77E080E090E00E94CC
:1024A0000C041F910F9108950FB6F8940F92E82F26
:1024B000FF27FE2FEE2790819083C59A0000C598D4
:1024C0000F900FBE8093EC010895BD9A8091EC01AE
:1024D0000E945412089521E030E002C0220F331F01
:1024E0008A95E2F78091EC01822B0E9454120895A4
:1024F00021E030E002C0220F331F8A95E2F72095D9
:102500008091EC0182230E9454120895A0912F0221
:10251000BB27FD01EE0FFF1FEE0FFF1FE75EFD4F14
:102520008083618342832383CD01019665E070E05F
:102530000E94321B282F80932F02809118022817A7
:1025400049F4822F9927019665E070E00E94321BC2
:102550008093180208958093D8016093ED01409311
:10256000D90108951F93182F80912D02882319F403
:10257000812F0E94CD1A81E090E002C0880F991F40
:102580001A95E2F7809520911702282320931702CD
:102590001F9108951F93182F80912D02882319F4FD
:1025A000812F0E94DB1A81E090E002C0880F991F02
:1025B0001A95E2F720911702282B209317021F91FA
:1025C0000895CF93DF93C82FDD27C0FF04C080E0BC
:1025D0000E94DB1A03C080E00E94CD1AC1FF04C034
:1025E00081E00E94DB1A03C081E00E94CD1AC2FF85
:1025F00004C082E00E94DB1A03C082E00E94CD1A70
:10260000C3FF04C083E00E94DB1A03C083E00E9482
:10261000CD1ADF91CF910895CF93DF93C0E0D0E042
:102620008091170299270C2E02C0959587950A94E0
:10263000E2F780FF04C08C2F0E94DB1A03C08C2FAE
:102640000E94CD1A2196C430D10551F7DF91CF9168
:10265000089580912F02809318020E940C1310920B
:102660002D0208951F93182F0E94E91A10922F022D
:1026700010921802112351F020E034E040E050E0C5
:1026800068E473E184ED91E00E94C5081F9108950C
:1026900086E90E944A05E091180280912F02E8170E
:1026A00019F410922D0245C0FF27EE0FFF1FEE0F09
:1026B000FF1FE75EFD4F808180932D0200E010E058
:1026C000802F0E94CD1A0F5F1F4F04301105C1F7F4
:1026D00080911802A82FBB27FD01EE0FFF1FEE0F00
:1026E000FF1FE75EFD4F83818F3F11F08150838391
:1026F000128180912D02843009F469C0853060F424
:10270000813009F449C08130A0F0823009F452C010
:10271000833009F062C187C0863009F4CEC08630AC
:1027200008F4A3C0873009F4F9C0883009F055C116
:1027300027C18091D901882329F10E942D1520916C
:10274000D801EFE32E9F90011124442755270E94C2
:10275000451B6F33710581059105A0F46091ED0172
:10276000662321F021E04091D90107C08091170232
:10277000882331F421E041E061E084E00E94861288
:1027800010922E0280912E028F5F80932E026FE3B3
:1027900070E080E090E00BC081810E94E1126FE365
:1027A000169FB0011124882777FD8095982F0E94ED
:1027B0000C041BC181810E94E1128FE3189FC001AC
:1027C00011247C010027F7FC0095102F21C080E028
:1027D0000E94E1128FE3189FC00111247C010027A1
:1027E000F7FC0095102FC801B7010E940C048091DE
:1027F0002D02882309F44FCFE0911802FF27EE0F36
:10280000FF1FEE0FFF1FE75EFD4F81810E94E11267
:10281000C801B7010E940C0480912D02882309F49D
:102820003ACF80E01FC080E00E94E1128FE3189F42
:10283000C00111247C010027F7FC0095102FC8016E
:10284000B7010E940C0480912D02882309F423CF44
:10285000E0911802FF27EE0FFF1FEE0FFF1FE75E4C
:10286000FD4F81810E94E112B5C080E00E94DB1A19
:10287000C12FDD278FE390E09C01C29FC001C39F61
:10288000900DD29F900D11247C010027F7FC00953C
:10289000102FDD24C801B7010E940C0480912D0285
:1028A000882391F18D2D0E94CD1AD3948D2D0E94F5
:1028B000DB1A33E0D31671F727C083E00E94DB1ADE
:1028C000C12FDD278FE390E0FC01CE9FC001CF9F99
:1028D000900DDE9F900D11247C010027F7FC0095E0
:1028E000102F63E0D62EC801B7010E940C0480911E
:1028F0002D02882349F08D2D0E94CD1ADA948D2D5A
:102900000E94DB1ADD2079F78FE390E0C89FB001C9
:10291000C99F700DD89F700D112445CF80E00E9493
:10292000DB1A8FE3189FC00111246C01EE24D7FC41
:10293000E094FE2C10E0C701B6010E940C048091C7
:102940002D02882349F0812F0E94CD1A1F5F812F0D
:102950000E94DB1A133079F713E0C701B6010E9419
:102960000C0480912D02882309F495CE812F0E94BA
:10297000CD1A1150812F0E94DB1A1123B1F1EDCF36
:1029800080E00E94DB1A81E00E94DB1A82E00E9454
:10299000CD1A83E00E94CD1A8FE3189FC001112445
:1029A0007C010027F7FC0095102FC801B7010E9499
:1029B0000C0480912D02882309F46DCE80E00E94E2
:1029C000CD1A81E00E94CD1A82E00E94DB1A83E0DA
:1029D0000E94DB1AC801B701EACEAA0FBB1FAA0FDB
:1029E000BB1FA75EBD4FFD01138280912D0288237E
:1029F00009F451CE80911802282F3327F901EE0FE8
:102A0000FF1FEE0FFF1FE75EFD4F8381882309F054
:102A100042CEC901019665E070E00E94321B209110
:102A20002F0233278217930711F40E940C13809111
:102A300018029927019665E070E00E94321B80938E
:102A4000180229CE6093EE017093EF018093F0019C
:102A50009093F101409330020895809130028130CB
:102A600089F40E94FF029B01AC018091EE019091DC
:102A7000EF01A091F001B091F101280F391F4A1F19
:102A80005B1F10C00E94FF029B01AC018091EE0110
:102A90009091EF01A091F001B091F101281B390B49
:102AA0004A0B5B0BCA01B90108950E94FF02089509
:102AB0000F931F93CF93DF93FC01C189D289EDA9B6
:102AC000FEA909958C01892B49F4CF5BDF4FE88182
:102AD000F98160E072EC81E090E00995C801DF9136
:102AE000CF911F910F910895CF93DF93EC01EA816D
:102AF000FB810188F289E02D0FB6F8940F9264A54E
:102B000075A50F900FBE88279927DF91CF91089563
:102B1000CF92DF92EF92FF920F931F93CF93DF93A9
:102B2000EC018B017A0169018C819D8128853985B1
:102B30000FB6F8940F92198618860F900FBE2617BD
:102B4000370789F0232B21F0009711F00E947311B1
:102B50000115110509F1C8010E947611009729F4A9
:102B60008FEF9FEF1BC0672BB9F09D838C839983F8
:102B700088839B838A83800F911F9F838E83FD862A
:102B8000EC86DF86CE861B861A860FB6F8940F92E7
:102B9000198708870F900FBE80E090E0DF91CF91FA
:102BA0001F910F91FF90EF90DF90CF900895CF92FB
:102BB000DF92EF92FF920F931F93CF93DF938A01DF
:102BC000DA01CD90DD90ED90FC902C2DFC01C189B7
:102BD000D289F1E067307F0709F464C081E0683092
:102BE0007807ECF491E06330790709F44AC0A1E07A
:102BF00064307A0754F4B1E061307B0799F1E1E089
:102C000062307E0709F0CCC030C0F1E065307F074C
:102C100009F442C0665071400CF041C03AC091E0E6
:102C20006B30790709F4A8C0A1E06C307A0754F43E
:102C3000B1E069307B0709F441C06A5071400CF083
:102C400076C033C0F1E06D307F0709F49FC081E0AA
:102C50006D3078070CF495C091E06E30790709F07B
:102C60009FC099C0CF5BDF4F5FC0CD5BDF4FE88176
:102C7000F9810995D8016D937D938D939C9313975A
:102C800036C1CB5BDF4FE881F9818C2D09958C0132
:102C900030C1C95BDF4F0BC0C75BDF4FF4CFC55BF3
:102CA000DF4F05C0C35BDF4FEECFC15BDF4FE88175
:102CB000F98109959927AA27BB2714C1C6FC03C02F
:102CC00000E010E011C0FE01B296268537854485EC
:102CD000558560857185CF010E9488158C01892BEF
:102CE00019F4EBADFCAD0995C7FE10C00115110537
:102CF00009F0FFC0FE01709626853785448555850D
:102D000060857185CF010E9488158C010115110520
:102D100009F0EFC0CF5ADF4F8FE39FEFAFEFBFEF68
:102D2000C822D922EA22FB22E881F9815DC0CD5A6E
:102D3000DF4FE881F981C355D04009959B01AC0173
:102D4000D8016D937D938D939C9313978CA59DA52E
:102D5000892B31F42064F80120833183428353832B
:102D60008A8D9B8D892B09F0C2C0F80180819181E9
:102D7000A281B3818068B7C0C886D986EA86FB86FF
:102D8000B6C088859985AA85BB85ACC0CC86DD8612
:102D9000EE86FF86ACC08C859D85AE85BF85A2C0C2
:102DA000FB01EF50F140E931F10540F4EA5BFF4FE0
:102DB000EE0FFF1F0590F491E02D09940FEF1FEF28
:102DC00098C088819981AA81BB81222311F08064F7
:102DD00022C08F7B20C088819981AA81BB8186FF18
:102DE00027C021C0EDADFEADC701B60109954FCF9B
:102DF000EF96E881F9810995F801608371838283F8
:102E0000938375C088819981AA81BB81222311F0A7
:102E1000806801C08F7788839983AA83BB8367C04A
:102E2000888187FF05C081E090E0A0E0B0E05AC053
:102E3000D8011D921D921D921C92139758C0CB5A17
:102E4000DF4FE881F981822F21CFC95ADF4F2FCF81
:102E5000FE0170962685378544855585B601CF01DC
:102E60000E9488158C01892B09F043C0EBADFCADA5
:102E700009953FC0888D998D33C0FE01B296268595
:102E8000378544855585B601CF010E948815FFCE50
:102E90008AA59BA525C00FB6F8940F92DD8ECC8E27
:102EA0001AC08C8D9D8D1CC00FB6F8940F92DF8ECA
:102EB000CE8E11C08E8D9F8D13C00FB6F8940F92D9
:102EC000DFA6CEA608C08EA59FA50AC00FB6F894AF
:102ED0000F92D9AAC8AA0F900FBE09C088A999A9B4
:102EE000AA27BB27F80180839183A283B38300E0E4
:102EF00010E0C801DF91CF911F910F91FF90EF90EB
:102F0000DF90CF900895CF92DF92EF92FF920F93D0
:102F10001F93CF93DF936C018A01FC01C189D28991
:102F200083E0E82EF12CE422F522E114F10481F093
:102F300028E330E048E250E060E470E0CE014096E3
:102F40000E948815892BA1F4F1E0EF16F10499F0A5
:102F500020EF30E040ED50E060E071E0CE0182967D
:102F60000E948815892B39F08C899D890E947311E4
:102F70000FEF1FEF2CC086E090E00E9476110097C3
:102F800039F48C899D890E9473118EA19FA1EECF87
:102F90000070107C288139814A815B810050104883
:102FA00011F42F7701C02068288339834A835B831B
:102FB0008C01FC0111821082D382C282158214829C
:102FC000F1E0EF16F10419F0EBADFCAD0995C80185
:102FD000DF91CF911F910F91FF90EF90DF90CF90F5
:102FE0000895CF93DF93DC01EC01EA81FB81C18975
:102FF000D28901978E5F9F4F18F08FEF9FEF19C016
:10300000CD010E94731120E030E040E050E060E02C
:1030100070E0CE0140960E94881520E030E040E04C
:1030200050E060E070E0CE0182960E94881580E05A
:1030300090E0DF91CF910895CF92DF92EF92FF92CF
:103040000F931F93CF93DF937C016A01EC0160968D
:103050000FB6F8940F928A859B85860F971F9B87E2
:103060008A8713C0F70181AD92ADFC010995F70184
:103070004485558566857785CE0140960E94FE077A
:10308000892B51F40FB6F8940F920A851B850F9087
:103090000FBEC016D10630F3C801DF91CF911F914A
:1030A0000F91FF90EF90DF90CF9008956F927F92F5
:1030B0008F929F92AF92BF92CF92DF92EF92FF9248
:1030C0000F931F93CF93DF93CDB7DEB722970FB641
:1030D000F894DEBF0FBECDBF4A015901FC01E18863
:1030E000F288A0E16A2E712C6E0C7F1CF3018085A2
:1030F0009185892B21F4FFEFCF2EDF2E9BC0611528
:10310000710549F440E050E060E070E0C7010E94C2
:103110001C186C018FC0F70180819181A281B3815D
:103120009C01AD01E9E05695479537952795EA95BD
:10313000D1F721702A8327E0B695A79597958795B3
:103140002A95D1F7817089830FB6F8940F92F30115
:10315000428553850F900FBE8B0160E070E0CC2458
:10316000DD2450C09A01260F371FF301868597850D
:103170002817390778F044855585C7010E941C1827
:10318000AC01F301848595858417950708F452C036
:1031900060E070E0A114B10419F0F801849102C05C
:1031A000D8018C91B981B13069F48A3081F4EA8117
:1031B000E13019F0F2E0F98303C082E08A83898369
:1031C0008DE00AC09981923011F4A1E0A9830F5FCC
:1031D0001F4F0894C11CD11CD301ED91FC91119794
:1031E00081931196FC93EE932D913C91F30186818E
:1031F00097812817390721F48481958191838083F1
:103200006F5F7F4FC814D9040CF4ACCF6115710502
:1032100089F00FB6F8940F92F30182859385860F9B
:10322000971F938782870F900FBEF70181AD92ADF4
:10323000FC010995C60122960FB6F894DEBF0FBEB9
:10324000CDBFDF91CF911F910F91FF90EF90DF9055
:10325000CF90BF90AF909F908F907F906F90089588
:1032600021E030E0FC01828193810E94561808958C
:1032700020E030E0FC01828193810E94561808957D
:10328000AF92BF92CF92DF92EF92FF920F931F9374
:10329000CF93DF937B015A01EC01EA81FB81018925
:1032A0001289E801A296688579856115710519F47E
:1032B0008FEF9FEFA1C0E114F10461F42E853F85EB
:1032C0004C855D85CE010E948815E801EBADFCAD13
:1032D00009951AC00FB6F8940F926A857B850F90F6
:1032E0000FBE6115710599F4F80183AD94ADFC0131
:1032F0000995F8014085518562857385CE01409618
:103300000E94FE07892B31F380E090E075C0D70161
:10331000F801808187FF35C0CC24DD24EE24FF2412
:103320005AE02BC0E616F70609F44FC0EA81FB818C
:103330004191FB83EA832A813B818E819F812817FB
:10334000390721F48C819D819B838A834D3011F054
:103350004A3051F4F80184A9882311F0841751F4FC
:10336000F80144AB5D9303C0F80114AA4D9308948F
:10337000C11CD11C0894E11CF11CCA14DB0490F29E
:1033800021C06B01A616B70608F4650140E050E0C5
:10339000D70114C0EA81FB8181918C93FB83EA837E
:1033A0002A813B818E819F812817390721F48C81E6
:1033B0009D819B838A834F5F5F4F11964C155D05FE
:1033C00049F77601E114F104B1F00FB6F8940F92C9
:1033D0008A859B858E199F099B878A870F900FBED0
:1033E0002A853B858C859D852817390720F4E801BF
:1033F000EBADFCAD0995C601DF91CF911F910F9107
:10340000FF90EF90DF90CF90BF90AF900895CF9353
:10341000DF93DC01EC01EA81FB81309719F08D919B
:103420009C910995DF91CF910895EF92FF920F93B0
:103430001F93CF93DF93EC017B018A01EC81FD8127
:10344000309719F480E090E005C060E070E080E023
:1034500090E0099519830883FB82EA82DF91CF917E
:103460001F910F91FF90EF900895CF93DF93EC01A0
:10347000EC81FD81309719F48FEF9FEF05C060E07C
:1034800070E081E190E00995DF91CF910895CF93AD
:10349000DF93EC01EC81FD81309719F48FEF9FEF02
:1034A00005C060E070E082E190E00995DF91CF9186
:1034B00008950F931F93CF93DF93CDB7DEB7249773
:1034C0000FB6F894DEBF0FBECDBF8C017C836B833B
:1034D000FC01248135812115310519F48FEF9FEF0F
:1034E00017C0BE016F5F7F4F80E290E0F901099540
:1034F000009771F4F80124813581BE016D5F7F4F23
:1035000081E290E0F9010995009711F489819A818F
:1035100024960FB6F894DEBF0FBECDBFDF91CF91DA
:103520001F910F9108950F931F93CF93DF93CDB702
:10353000DEB724970FB6F894DEBF0FBECDBF8C0167
:103540007C836B83FC01248135812115310519F4BD
:103550008FEF9FEF17C0BE016F5F7F4F88E190E054
:10356000F9010995009771F4F80124813581BE01B4
:103570006D5F7F4F89E190E0F9010995009711F4A3
:1035800089819A8124960FB6F894DEBF0FBECDBF15
:10359000DF91CF911F910F910895882321F0813001
:1035A00011F0823019F40E9478120895833011F4DA
:1035B0000E9478120895882321F0813011F0823022
:1035C00019F40E946B120895833011F40E946B125B
:1035D00008950E94651280E00E94CD1A81E00E9449
:1035E000CD1A82E00E94CD1A83E00E94CD1A089580
:1035F000DC0140FF03C001C06D936D934250504009
:10360000D8F70895FB01DC018D910190801911F428
:103610000020D1F7990B0895FB01DC0101900D9278
:103620000020E1F70895629FD001739FF001829F0F
:10363000E00DF11D649FE00DF11D929FF00D839F41
:10364000F00D749FF00D659FF00D9927729FB00DDE
:10365000E11DF91F639FB00DE11DF91FBD01CF01F1
:103660001124089597FB092E07260AD077FD04D070
:103670002ED006D000201AF4709561957F4F0895E2
:10368000F6F7909581959F4F0895A1E21A2EAA1BF7
:10369000BB1BFD010DC0AA1FBB1FEE1FFF1FA21702
:1036A000B307E407F50720F0A21BB30BE40BF50BFF
:1036B000661F771F881F991F1A9469F76095709588
:1036C000809590959B01AC01BD01CF010895AA1B87
:1036D000BB1B51E107C0AA1FBB1FA617B70710F0FD
:1036E000A61BB70B881F991F5A95A9F7809590952F
:1036F000BC01CD010895E199FECFBFBBAEBBE09AFE
:1037000011960DB20895E199FECFBFBBAEBB0DBAC5
:0E37100011960FB6F894E29AE19A0FBE089552
:10371E00722B00554152542D6563686F2061707095
:10372E006C69636174696F6E210A006574686572F5
:10373E006E75740069646C65006D61696E00FF00E2
:10374E00000000DD09000075617274300000000099
:10375E0005000000000058015815D71540193819FA
:10376E0030198317F11774150000000000000000D7
:10377E00000000000000000000000000000000003B
:10378E00000000000000000000000000000000002B
:10379E0000000000000000000000000000640D3B6F
:1037AE000D840C860C890D640CE40DEE0CB20C46E7
:1037BE000B600E630B940E740BE80B7E0B240E4DF8
:1037CE000C00000000EE0E000000005A0F0000007A
:1037DE0000BE0F0100020003000000000000000008
:0A37EE00000000004C4544000F01EC
:00000001FF
